:020000040000FA
:060000000219FD0200B32D
:03002B0002008D43
:03005B0002028618
:030073000200A0E8
:100080000406080C10182030406080A0C0C0D0C00A
:10009000E0C2CF0541E52360021523D0E0D0D03285
:1000A000C2AF53E67F7592FA7593FFC22053917FDA
:1000B000D2AF32C0D0C0E0C0F0D2D35388EFA88A0C
:1000C000A98C758A00758C0043881030331FE8C4F2
:1000D000540FFAE9C454F04AFAC3132AFAC3E833B6
:1000E000F8E933F9E82AFAE93403FB213630320F14
:1000F000C3E833E933FAE82AFAE93400FB21363061
:100100003115E875F056A4AAF0E975F056A42AFA5C
:10011000C5F03400FB2136E875F02BA4AAF0E97590
:10012000F02BA42AFAC5F03400C313FBEA13FAC378
:10013000EB13FBEA13FAC3EB94095006C3EB9403E9
:10014000501A0522E52270021522C3E522940A50B6
:1001500002417C7552007A007B00414EE52260022C
:1001600015223035067C007D042176AC31AD32306D
:100170003A04AC33AD34C3EA9CFAEB9DFB9208AE73
:100180005EAF5F303A425007203409D234219430B8
:100190003402C234303404AE60AF61203902B2346C
:1001A000C3EA33FAEB33FBA208500AEAF42401FA5B
:1001B000EBF43400FBC3EA9428FAEB9400FB5014F0
:1001C00078007A007B0021D4A208500878007A00D9
:1001D0007B00412AE52554036019202A16E55BF9C6
:1001E000EB7007C3E99A4002E9FAE53CC42AFAEB4E
:1001F0003400FBEA8EF0A4F9AAF0EB8EF0A42AFA00
:10020000C5F03400FBC3EB13FDEA13F80FEF1460E5
:1002100004C3E833F8C3E933EA33FAEB33FBDFED29
:10022000EB30E20678FF7AFF7B038852D230C3E8D6
:1002300094404002D221C3E559FC955A4003AC5A80
:10024000C3EC95525008EC75F004A4FAABF0EAF454
:10025000F8EBF45403F98854895575230AE55830AE
:10026000E10DD0F0D0E0D0D053F7DF43F74032D0EB
:10027000F0D0E0D0D053D8FE43DA013275230AD053
:10028000F0D0E0D0D032C0D0C0E0D2D38554FB85CE
:1002900055FC85555853F7BF53DAFEC3E552940118
:1002A000400575530041B2E5532401F553500375E1
:1002B00053FF53F7DF53D8FED0E0D0D0327901801E
:1002C0001479038010790A800C791E800879648083
:1002D0000479C880007817E4D5E0FDD8FAD9F62271
:1002E0007A147B7880127A107B8C800C7A0D7BB428
:1002F00080067A0B7BC880007902E4C293D5E0FDCA
:10030000D292D293D5E0FDC293D5E0FDC292D293B2
:10031000D5E0FDE920E004D290D29130E004D294FF
:10032000D295E562D5E0FDE920E002C29130E0021D
:10033000C2957496D5E0FDD9C1EAF8D5E0FDD8FBA9
:10034000DBB6C2932278FFC22120283D202912D299
:1003500021C3E548940A4009C3E55294405002C2C3
:100360002179A1E76023E548601F74FF8548F08488
:10037000853FF030290375F005A4F8C5F0600278D8
:10038000FFC3E8955B5002A85B885A22C3E54794F7
:10039000E4E5489400E55A500314619D046002F5B9
:1003A0005A2275E89022055CC3E55C94084055E547
:1003B000E820ECF2A8BDA9BE755C00E9FA79A0E7D7
:1003C0006041EA7006E55D6018800CC3E8955D60E9
:1003D0000EE55D5005600A1480070460FA8002E5AE
:1003E0005DF55DC394F6401B7559C0C39406401378
:1003F000755980C39406400B755940C39406400359
:1004000075590022E5592410500274FFF5592274E1
:100410003279A687F0A4C5F0A2F733F8C3E895595E
:100420004002A859885B227547007548F022C2AF88
:1004300075C800A8CCA9CDAA4130CF010A75C8045F
:10044000D2AFAB42AC4388428943C3E89BF8E99CF6
:10045000202808F9302C02A13A8197AD448A44F94A
:10046000EA9DFA600478FF79FFAE45AF468B458C74
:1004700046A842A943C3E89EF8E99FF9C3E548139B
:10048000FBE54713FAE82AF547E93BF548500675BE
:1004900047FF7548FF81E1AA47AB48AC47AD487EAE
:1004A000047F02C3EB9404400A1E1FC3EB94084070
:1004B000021E1FC3ED13FDEC13FCDEF7C3EA9CFA2A
:1004C000EB9DFBEF6009C3E913F9E813F8DFF7EAE6
:1004D00028FAEB39FB8A478B4850067BFF8B478B0A
:1004E00048C3EB94025002D22C3028047F03A10CA5
:1004F0007892E6FFC3E53D948240110FC3E53D9439
:10050000A040010FC3EF940640027F057E02E5483C
:10051000C4540FF9E548C454F0F8E547C4540F2813
:10052000F8C3E89EFAE99400FB4009C3EA9401EBA2
:10053000940050047A01E4FBA186AA47AB48EBC4BF
:10054000FEEAC4540F4EFCC3EA9CFAEB9400FBC3D2
:10055000E813C313F8EA28FAEB3400FB8A478B4808
:10056000C3EB94024002C22C7802EBC4FE7B00EA8B
:10057000C4540F4EFAC3EA98FA4005C394015002DE
:100580007A017892E6FF30200280FB854E92854FFB
:1005900093D22043E680C3E49AF8E49BF9302C021E
:1005A000C111E8FAE9FBD3E913FDE813FC884E8991
:1005B0004FC3EF94036037EF20E00CE82CF8E93DDF
:1005C000F9ECFAEDFB8013E828F8E939F9C3E824DF
:1005D00001F8E93400F97AFF7BFFC3EF9403400E82
:1005E0008A508B51884A894B8C4C8D4DC14588501F
:1005F00089518A4A8B4B8C4C8D4D3028127550F0A6
:100600007551FF754CF0754DFF754EF0754FFFC17C
:1006100045E8FAD3E813FC884EC3EF94036020EF5B
:1006200020E007E82CF8ECFAC131E8282401F87A38
:10063000FFC3EF940340088A50884A8C4CC1458818
:10064000508A4A8C4C302002C145753A02D2204370
:10065000E680E52554036034A847A948C3E913F9A7
:10066000E813F8C3E913F9E813F8302804E9244043
:10067000F9C2AF53E67F759100C3E498F594E4990D
:10068000F595759104D22043E680D2AF22D222752F
:100690004900752000302B03752040800ED2227552
:1006A0004900752040302B03752000780179012026
:1006B0002C20E52554036002C2227914E548C313B7
:1006C000700104F8C3941440027814302804781B95
:1006D000791B202010E549600C302803D53A04D25C
:1006E00024E14DD14D0549E59B5440B52002E13749
:1006F00030280908C3E899400118C1D220220A080D
:10070000C3E8994002C1ABC1D2C222C2AF53E67F57
:10071000759100302C127594007595FE759104D278
:100720002043E680D2AFC1ABAE47AF48C3E49EF5ED
:1007300094E49FF595E11CC3E53994015002C1ABE7
:10074000302202C1ABD802E14BC1D2C224C2AF53A6
:10075000E67F759100855094855195759104854A81
:1007600092854B93D22043E680D2AFE525540360B7
:10077000072029020539801030240D202B0A202261
:100780000715811581020EB4227800302105302230
:10079000027801E53D75F007A4F9E5F028F5F0E9E8
:1007A000A2F013A2F113A2F213F53DC39478500303
:1007B000753D78C3E53D953E400BD223C291C2936F
:1007C000C29575D57F30200280FB854C92854D9374
:1007D000D22043E68022203815C2AFC293C290D205
:1007E00091D29575D56FD2AF759F200208DBC2AF4D
:1007F000C293C294D295D29175D57ED2AF759F2007
:1008000001DB203815C2AFC295D29375D57BC2905B
:10081000D291D2AF759F300208DBC2AFC291D293A2
:1008200075D57BC294D295D2AF759F100208DB209C
:100830003814C2AFC291C294D295D29375D57BD2EF
:10084000AF759F1001DBC2AFC295C290D291D29317
:1008500075D57BD2AF759F3001DB203815C2AFC292
:1008600093D29175D57EC294D295D2AF759F200256
:1008700008DBC2AFC293D29575D56FC290D291D228
:10088000AF759F200208DB203814C2AFC295C29218
:10089000D293D29175D57ED2AF759F30803DC2AFD5
:1008A000C291C292D293D29575D56FD2AF759F1077
:1008B0008029203814C2AFC291D29575D56FC292EB
:1008C000D293D2AF759F108012C2AFC295D29175EC
:1008D000D57EC292D293D2AF759F30C22322C291ED
:1008E000C293C295C291C293C29575D57F2278807A
:1008F00076FF0876FF0876FF0876FF0876FF087611
:10090000FF0876090876FF087601788C760108766C
:10091000FF0876FF0876FF0876FF0876FF08760363
:100920000876FF0876FF0876FF0876250876D00857
:1009300076280876500876040876FF08760208764E
:10094000FF08767A0876FF0876010876010876FFB8
:100950000876FF08760008760022FA75F00CA4AB42
:10096000F0EAC333F8740133F9E8C333F8E933F933
:10097000E8C32BF8E93400F9227888E6C39403D25F
:100980003A5002C23AC238E630E102D238A2389276
:10099000397886E6149000809378A6F67886E6F596
:1009A0003FC394025003753F02789CE6753EFFB446
:1009B0000203753EA0B40303753E827896E6315A71
:1009C00088318932789EE6315A883389347897E6BF
:1009D000315A8835893611DE223035117A007B0094
:1009E0007CFF7D007E0051408B5F8A5E22303A2280
:1009F0007896E6FA7B00789EE6FC7D00C3EA33FA3F
:100A0000EB33FBC3EC33FCED33FD7E0A51408B61CD
:100A10008A607896303A02789EE6FA7B007897E60C
:100A2000FC7D007E00303A10C3EA33FAEB33FBC39F
:100A3000EC33FCED33FD7E0A51408B5F8A5E22224F
:100A4000C3EC9EFCED9400FDC3EC9AFCED9BFDC352
:100A5000EC9423ED940050047C237D00C3EC94FFC0
:100A6000ED940140047CFF7D017BFF0B7A000AEAD4
:100A70007009C3EC33FCED33FD416BEC8AF0A4AE9E
:100A8000F0ED8AF0A42E947C40E4EAF460DD22D2FA
:100A90003531D91202C97A007B007C101202C1E5FF
:100AA000522AFA74003BFBDCF37C04C3EB13FBEA31
:100AB00013FADCF7FFEB60027FFFC23531D92278F1
:100AC000A5E6F95403D2867002C286E9540CD28797
:100AD0007002C287E95430D2967002C296E954C0BF
:100AE000700022E5EF20E6037520000520903FFF0F
:100AF000E520146006901DFF1460009304600375E8
:100B0000EF127597DE7597AD7581C043FF801202B5
:100B1000BD75EF0275A90011DE75803F75F1F075A6
:100B2000A4C075803F75D4FF75900075F27F75A5E0
:100B30007F75900075D57F75A60175E34075E2025B
:100B4000C291C293C2951202CDC290D291C292D2EA
:100B500093C294D2951202BDC291C293C29511DE86
:100B6000E4F8F6D8FD11EED1EC7898866275300184
:100B7000C2AF1202D11202E01202C91202E6120240
:100B8000C91202EC1202C951BFC2AF78FA79FA3029
:100B90008507D9FBD8F7021C00317931D9789886BE
:100BA0006211DE75E405758811758E047589097505
:100BB000C80475910475D84075D90875F782759E7B
:100BC0000075960275DA4A75DB0075A82175E69006
:100BD00075F310759B80759D0075D12C75BC58758B
:100BE000BB1075E88075B2011202BDD2AF753C0032
:100BF000C2301202D1C2317522001202CDC3E522E9
:100C0000940A4024D231C2327522001202CDC3E5CB
:100C100022940A4013D232C2337522001202CDC38D
:100C2000E522940A4002D2331202C1203003020BA3
:100C300089C2AF1202E01202E01202E0D2AF120249
:100C4000D1303A0281D31202C1788CE6C3940150AC
:100C50000281D3E530C39401500281D37F02D235A3
:100C600031D91202CDC2AFC23531D9AE52C3E5522D
:100C7000947FD2AF405D1202BDC2AF1202F2D2AF7A
:100C8000DFDC518FC3EF7897F61202D1F126F1C85D
:100C90007F0AD23531D91202CDC2AFC23531D9AEB9
:100CA00052C3E552947FD2AF50E61202BDC2AF12DA
:100CB00002E01202C51202E0D2AFDFD6518FEF245C
:100CC000037896F61202D1F126120FF71202CD31F7
:100CD000D961891202CD7801303A027805C3E55214
:100CE0009840028141C2AF1202F21202F21202F2E5
:100CF000D2AF1202D1753000E4F537F5380537E58B
:100D000037F4703E0538789AE67819146012783214
:100D100014600D787D14600878FA1460037538004B
:100D2000C3E53898401C11DE1202BD153875370036
:100D300078998662C2AF1202F2D2AF7898866212B8
:100D400002CD1202C5E523700261897801C3E55224
:100D50009840AA1202CDE5237003020B89C2AF119D
:100D6000DEE4D2AFE4F55CF524F525F53D755C08CD
:100D70001202BD1203A2E5E820ECFBA8BDA9BEE962
:100D80007001F8885D1203A6755C08C2AF7559FF43
:100D900012040F855B59855B5AD2AF303A07C238CF
:100DA000303402D238D228753900118711B21204BA
:100DB0002712042E12042712042E12042712069D55
:100DC0001207891207D612042E12068D202C031248
:100DD0000345302C0312038C120789110212042ED2
:100DE00012069D120789112F12042E12068D12076A
:100DF00089115A12042E12069D12078911871204B6
:100E00002E1203A212068D12078911B21203A61226
:100E1000042E302827855B5979187A0CC3E5399957
:100E2000400EC228D2298A3B855B59855B5A800CCB
:100E3000C3E55294014003020DBDC1BC30291C2002
:100E40002B19E53B147006C229D22AA1BDF53BC37C
:100E5000E55294014003020DBD8061753C0078FAB3
:100E600079A4E760027803C3E55398504FE5236007
:100E70004B303A17203805203407800F3034028079
:100E80000A202B07D22B855B59A1EB78F0302B057C
:100E9000855B597820C3E548985003020DBD302B7F
:100EA0001BC22BC238303402D238D229753B12858E
:100EB0005B59A1BD053CE5526002C1BF753C00C253
:100EC000AF11DE752400752500D2AF1202CD11DE00
:100ED00078A4E6600CC290D291C292D293C294D20E
:100EE00095C3E53C94044002618981F8901A0D781D
:100EF00020F15FE520B4550AA3F15FE520B4AA0212
:100F0000800611EEF126801D901A0378807B0AF18D
:100F10005FA308DBFA901A0F788C7B1AF15FA308A5
:100F2000DBFA901A2922C2AFF19EF178901A007470
:100F300010F164A37401F164A37420F164901A03A6
:100F400078807B0AF163A308DBFA901A0F788C7B18
:100F50001AF163A308DBFAF1B1F18F901A2922E4A8
:100F600093F622E6438F01538FFD75EF0275B7A507
:100F700075B7F1F0538FFE22438F02438F0175EF57
:100F80000275B7A575B7F1901A0DF0538FFC22903A
:100F90001A0D7455F164901A0E74AAF164227A3015
:100FA00079D07820901A40F15FE520F709A3DAF7AD
:100FB000227A3079D0901A40E7F16409A3DAF92255
:100FC0007C051202D1DCFB22C2AF1202E01202E663
:100FD0001202EC1202F21202C51202E01202E61232
:100FE00002EC1202F21202C51202E01202E6120232
:100FF000EC1202F2D2AF22C2AF1202F21202EC12D3
:1010000002E61202E01202C51202F21202EC120211
:10101000E61202E01202C51202F21202EC1202E61D
:061020001202E0D2AF2233
:1019FD00020AE3100120FFFFFFFFFFFF09FF01FFB8
:101A0D0055AA01FFFFFFFFFF03FFFFFF25D0285061
:0D1A1D0004FF02FF7AFF0101FFFF0000FF40
:101A400023455F4C5F3030232020202020202020A1
:101A500023424C48454C492445464D3842313023B9
:101A60002020202020202020202020202020202076
:101C0000C2AFC2D37597DE7597AD7581C075A90057
:101C100043FF80752438752503B1C875EF0243F181
:101C20002053A4DFD28575D4FF75E3407DFA780395
:101C300079E67C10752200752300901DD57B067512
:101C400024987525013085028145208508D8FBD967
:101C5000F9DCF781B7308508D8FBD9F9DCF781B713
:101C6000B188E493A3C39A6004DDC381B7DBDBB121
:101C70007A6002812E7B08E493FAA3B15BDBF87AE9
:101C800030B15B752200752300B17AEAFCEBFDC32D
:101C9000ED94FE400EB17A8A278B28ED30E0048A5D
:101CA000828B83B17A7AC270D8C3ED94FE601350F0
:101CB000CEBD0023EC60097520007521FF020000F5
:101CC0008100A827A9280809D804D90281D4B17EA7
:101CD000EAF281C80D81A3C3ED94035047EDA2E061
:101CE00092007AC5C3E5829400E583941C5092204B
:101CF0000010438F02438F0175B7A575B7F1F0301F
:101D0000001DA827A9280809438F01538FFDD80477
:101D1000D902A11FE275B7A575B7F1F0A3A10E53C3
:101D20008FFC817F7AC1BD030CE493A3FAB13FDC41
:101D3000F8B137817F8181AA22AB23B15BEBFAEA4C
:101D40006222752608C3E52313F523E52213F52245
:101D500050066323A0632201D526EAB1C8B1C87535
:101D6000260AEAF4200102D285300102C285B1C8F8
:101D7000C3134002C201D526EB22B17EEAFB2085C7
:101D800002A17E308502A183752608AE24AF25C34B
:101D9000EF13FFEE13FEB1CCB1C8C3EA13308502D6
:101DA0004480FA30E703632201C3E52313F523E5FA
:101DB0002213F52250066323A0632201D526D9E51C
:101DC0002265236523F52222AE24AF250E0FDEFE09
:101DD000DFFCD20122424C48656C6934373163E83C
:031DE000B1060148
:00000001FF
